:100000000C9461000C947E000C947E000C947E0095
:100010000C947E000C947E000C947E000C947E0068
:100020000C947E000C947E000C947E000C947E0058
:100030000C947E000C947E000C947E000C947E0048
:100040000C94A9000C947E000C947E000C947E000D
:100050000C947E000C947E000C947E000C947E0028
:100060000C947E000C947E00000000002400270009
:100070002A0000000000250028002B0000000000DE
:1000800023002600290004040404040404040202DA
:100090000202020203030303030301020408102007
:1000A0004080010204081020010204081020000012
:1000B0000007000201000003040600000000000029
:1000C000000011241FBECFEFD8E0DEBFCDBF11E08E
:1000D000A0E0B1E0EEE3F4E002C005900D92A430A0
:1000E000B107D9F711E0A4E0B1E001C01D92AD3035
:1000F000B107E1F70E94A2000C941D020C940000CD
:10010000809102010E94CE01019781F4809100014B
:1001100061E00E94810168EE73E080E090E00E945F
:10012000FD008091000160E00E94810108958091AE
:10013000000161E00E9461018091020160E00E9483
:10014000610108950E9427010E9497000E9480008B
:10015000FDCF1F920F920FB60F9211242F933F9352
:100160004F935F936F937F938F939F93AF93BF93BF
:10017000209108013091090140910A0150910B0131
:1001800070910C01DA01C9010296A11DB11D672F02
:100190006A5F6D3730F06D57DA01C9010396A11D12
:1001A000B11D60930C018093080190930901A09305
:1001B0000A01B0930B018091040190910501A09177
:1001C0000601B09107010196A11DB11D80930401A4
:1001D00090930501A0930601B0930701BF91AF91E1
:1001E0009F918F917F916F915F914F913F912F914F
:1001F0000F900FBE0F901F901895EF92FF920F93E4
:100200001F937B018C018FB7F894409108015091A6
:10021000090160910A0170910B018FBF2FB7F8940B
:100220008091080190910901A0910A01B0910B0100
:100230002FBF841B950BA60BB70BE816F9060A0710
:100240001B0760F71F910F91FF90EF90089578942E
:1002500084B5826084BD84B5816084BD85B58260CB
:1002600085BD85B5816085BDEEE6F0E08081816069
:100270008083E1E8F0E0808182608083808181601A
:100280008083E0E8F0E0808181608083E1EBF0E052
:10029000808184608083E0EBF0E0808181608083F6
:1002A000EAE7F0E0808184608083808182608083DF
:1002B0008081816080838081806880831092C1000A
:1002C0000895282F30E0C90186569F4FFC01949174
:1002D0002A573F4FF9018491882391F0E82FF0E0ED
:1002E000EE0FFF1FE859FF4FA591B491662329F443
:1002F0008C91909589238C9308958C91892B8C9364
:100300000895482F50E0CA0182559F4FFC01249167
:10031000CA0186569F4FFC0194914A575F4FFA01DC
:1003200034913323D1F1222331F1233021F4809110
:1003300080008F7705C0243031F4809180008F7D5C
:100340008093800018C0213019F484B58F7704C0E1
:10035000223021F484B58F7D84BD0DC0263021F478
:100360008091B0008F7705C0273029F48091B000CC
:100370008F7D8093B000E32FF0E0EE0FFF1FEE586B
:10038000FF4FA591B491662329F48C919095892310
:100390008C9308958C91892B8C930895682F70E02D
:1003A000CB0182559F4FFC012491CB0186569F4F74
:1003B000FC0144916A577F4FFB019491992319F4F2
:1003C00020E030E038C0222331F1233021F4809145
:1003D00080008F7705C0243031F4809180008F7DBC
:1003E0008093800018C0213019F484B58F7704C041
:1003F000223021F484B58F7D84BD0DC0263021F4D8
:100400008091B0008F7705C0273029F48091B0002B
:100410008F7D8093B000892F90E0880F991F8458BA
:100420009F4FFC01A591B4918C9120E030E0842392
:0E04300011F021E030E0C9010895F894FFCFEB
:04043E0003000200B5
:00000001FF
